:100000000C9469000C9491000C9491000C94910054
:100010000C9491000C9491000C9491000C9491001C
:100020000C9491000C9491000C9491000C94A60BEC
:100030000C9491000C9491000C9491000C949100FC
:100040000C9424130C9491000C9449160C947B1678
:100050000C9491000C9491000C9491000C949100DC
:100060000C94860A0C949100000000090003020021
:10007000000405080000000000000000000000016E
:10008000020408102040800102040810200102042C
:100090000810204080400404040404040404020204
:1000A000020202020303030303030202030000002F
:1000B0000023002600290000000000250028002B56
:1000C0000000000000240027002A000096037709A2
:1000D000AB1611241FBECFEFD8E0DEBFCDBF12E0BC
:1000E000A0E0B1E0E6EDF0E302C005900D92A03E85
:1000F000B107D9F726E0A0EEB2E001C01D92A13110
:10010000B207E1F710E0C9E6D0E004C02197FE0194
:100110000E943418C636D107C9F70E94C7170C943D
:1001200069180C940000862F642F0C949114FC0124
:1001300081890E94FB1421E0892B09F420E0822FA1
:100140000895FC01DB0185E991E09183808312969B
:100150004D915D916D917C9115974283538364839A
:10016000758316968D919C91179797838683189621
:100170008C911897808719964D915D916D917C9126
:100180001C9741875287638774871D964D915D91B7
:100190006D917C915097458756876787708B5196F4
:1001A0008C915197818B8BE991E09183808352965A
:1001B0008C91828B0895EF92FF920F931F93CF93B0
:1001C000DF9326E040E855E260E070E084E795E0E8
:1001D0000E94F7150E94910D8DE794E00E94DF08C0
:1001E0008BE893E00E9421088BE893E00E942607A9
:1001F0008BE893E00E94710709E912E0C3EFD2E0B7
:100200007801F70161917F0170E0CE010E94F9064B
:1002100065E070E0CE010E9463061A8A6396FDE9EC
:10022000EF16F2E0FF0669F763E070E080EF92E01E
:100230000E94FB0C60910C0170E080EF92E00E9444
:10024000360D80EE92E00E947A0F61E084E00E9419
:10025000911461E08EE00E94911461E085E00E94BB
:10026000911461E086E00E94911461E089E00E94AF
:10027000911461E081E10E94911461E082E00E94AA
:10028000911462E0F80181918F010E949114F2E0D3
:100290000E391F07B1F761E084E00E94CD1470E0D1
:1002A00060E085E00E940B1470E060E086E00E9450
:1002B0000B1470E060E089E00E940B1460E081E1C3
:1002C0000E94CD1460E082E00E94CD14E2E7F4E0E9
:1002D0008CE794E02FE521938E179F07E1F7DF91DC
:1002E000CF911F910F91FF90EF9008950F931F935F
:1002F000CF93DF938B01EA01BC0185E00E940B14D0
:10030000B80186E00E940B14BE0189E0DF91CF9115
:100310001F910F910C940B1450E040E070E060E0EE
:1003200090E080E00C947601813041F028F082303A
:1003300069F0833091F008950C948C0150E040E016
:1003400070E060E08FEF90E00C94760150E040E0C8
:100350006FEF70E090E080E0F7CF4FEF50E070E09B
:1003600060E0F8CF8BE893E00E94710740E062E024
:100370008BE893E00E947F076EE071E08BE893E0EA
:100380000E94141741E060E08BE893E00E947F0731
:1003900062E774E08BE893E00E9414178BE893E027
:1003A0000C942B070E94591861E0892B09F04CC06E
:1003B00086E00E94CD148BE893E00E94710740E034
:1003C00065E08BE893E00E947F0766E371E08BE8CD
:1003D00093E00E94141741E062E08BE893E00E94F2
:1003E0007F076DE371E08BE893E00E94141761E0F2
:1003F00084E00E94CD148091080180930A016091ED
:100400000B0170E080EF92E00E94360D68EB7BE01C
:1004100080E090E00E949F1360E086E00E94CD148F
:100420008BE893E00E9471078BE893E00E942B0712
:1004300040E060E08BE893E00E947F0769E471E0B0
:100440008BE893E00C94141785E00E94CD148BE8A0
:1004500093E00E94710740E065E08BE893E00E9422
:100460007F0766E371E08BE893E00E94141741E098
:1004700065E08BE893E00E947F076AE571E08BE816
:1004800093E00E94141768EB7BE080E090E00E940C
:100490009F1360E085E00C94CD14AF92BF92CF9291
:1004A000DF92EF92FF920F931F93CF93DF937C0124
:1004B000FC0101900020E9F731978F01081B190B0F
:1004C000680120E1C21AD10880E1A82EB12C8091E8
:1004D00061048017110631F141E060E08BE893E0A0
:1004E0000E947F0762E671E08BE893E00E94141798
:1004F00066E970E080E090E00E949F1341E060E0D8
:100500008BE893E00E947F0701311105C4F4B70125
:100510008BE893E00E94141768EB7BE080E090E0AA
:100520000E949F1310926104DF91CF911F910F9150
:10053000FF90EF90DF90CF90BF90AF9008958091A3
:10054000610490E0E701C80FD91F8C159D052CF5BB
:1005500020916104822F90E00F96AE014E195F0941
:100560008417950734F069918BE893E00E941C177B
:10057000EFCF211106C06CED75E080E090E00E94A5
:100580009F136AEF70E080E090E00E949F138091DB
:1005900061048F5F809361049ACFCE018E199F0909
:1005A0008017910734F469918BE893E00E941C173F
:1005B000F4CFD0E0C0E0809161049801281B31099C
:1005C000C9019501281B390B2C173D07D4F260E2B5
:1005D0008BE893E00E941C172196EDCFCF93C82F94
:1005E0008BE893E00E9471078BE893E00E942B0751
:1005F00040E0CA3009F467C060E08BE893E00E94F5
:100600007F0763E771E08BE893E00E9414174AE0EC
:1006100050E06C2F8BE893E00E947C17C23009F405
:1006200060C008F042C06091060170910701C130BE
:1006300009F444C08CEF93E00E944D028BE893E0F4
:100640000E94710780910A01843020F48BE893E0C6
:100650000E942607ECEFF3E080E694E020E221938D
:100660008E179F07E1F780910A01843009F043C09B
:1006700040E062E08BE893E00E947F076EE071E06B
:100680008BE893E00E94141741E060E08BE893E070
:100690000E947F0762E774E08BE893E00E941417E2
:1006A0008BE893E0CF910C942B07C330F9F0609165
:1006B000000170910101C43009F0BCCF8CEF93E0D0
:1006C0000E946218B7CF61E08BE893E00E947F0739
:1006D00062E871E08BE893E00E94141768E973E028
:1006E000EDCF6091040170910501E8CF60910201A6
:1006F00070910301E3CFCF910895DC01FB019C9140
:100700008081981311C011969C9111978181981343
:100710000BC012969C9112978281981305C081E0BC
:1007200013962C919381291380E008950F931F93C2
:10073000CF9322E040E160910D018BE893E00E94AD
:10074000010788E793E00E94EC06E8E7F3E00BE995
:1007500011E011830083C1E0C28B85E693E00E9423
:10076000EC06E5E6F3E011830083C28B82E593E0BB
:100770000E94EC06E2E5F3E011830083C28B8FE375
:1007800093E00E94EC06EFE3F3E011830083C28B59
:1007900068E773E083EF92E00E94A10065E673E0F2
:1007A00086E093E00E94A10062E573E089E193E0B6
:1007B0000E94A1006FE373E08CE293E00E94A1002D
:1007C00080EF92E00E94610C40E16EE080EE92E0EA
:1007D000CF911F910F910C94570EFF920F931F937F
:1007E000CF93DF9390910A018091090198130E94A1
:1007F000B201C3EFD2E010E000E0CE010E947F061C
:10080000888582FF22C0CE010E94E8069A8989135A
:100810001CC060917104F801EC56FD4FF080E62F8A
:10082000F0E0EE58FB4FF08241E08BE893E00E944D
:100830007F076F2D8BE893E00E94B70780917104CA
:100840008F5F809371040E94B2010F5F1F4F639608
:100850000430110591F6809171048A30F1F463E25D
:1008600071E082E794E00E94D20110927104E2E705
:10087000F4E08CE794E02FE521938E179F07E1F7D2
:1008800090910A0180910801981739F0DF91CF917A
:100890001F910F91FF900C94B201DF91CF911F91A6
:1008A0000F91FF9008950F931F930E946E13009174
:1008B0006404109165042091660430916704601B04
:1008C000710B820B930B603177428105910578F0B3
:1008D0008091630481110BC010926D0410926E041C
:1008E00010926F041092700481E08093630480EE94
:1008F00092E00E94AD1290E090936B0480936A04A2
:1009000080EE92E00E94C70D282F30E030936904FA
:100910002093680420916A0430916B04232B09F41E
:1009200052C0882309F44FC08091E30280936D0484
:100930008091E40280936E048091E50280936F04BD
:100940008091E602809370041092630480EE92E03E
:100950000E94DD1280EE92E00E9420130E946E132E
:1009600060936404709365048093660490936704B5
:100970006DE674E08FE191E00E947D0380936C044A
:1009800081110DC081E00E94940168EB7BE080E062
:1009900090E00E949F131F910F910C948C01813065
:1009A000A9F482E00E94940168EB7BE080E090E093
:1009B0000E949F130E948C0180910A01833019F4D8
:1009C00084E080930A011F910F9108958230D9F736
:1009D00083E00E94940168E572E080E090E0D9CF66
:1009E000CF9384E795E00E94241518161906B4F4F5
:1009F00084E795E00E943E1580936004883609F4F0
:100A00006BC0ECF4833309F472C054F4813309F4FD
:100A100068C00CF06AC0843209F493C0CF91089585
:100A2000823609F452C024F48433C1F784E05AC0FA
:100A3000833609F478C0873689F782E043C082376D
:100A400009F43FC034F58F3609F441C0803709F40A
:100A500041C08D3619F764E670E080E090E00E94B6
:100A60009F13C0E084E795E00E942415181619062C
:100A70000CF05CC084E795E00E943E1580939703DC
:100A8000843281F3EC2FF0E0E856FC4F8083CF5F97
:100A9000E9CF853771F144F460E0833709F0BECFC8
:100AA00084E0CF910C94CD14863781F160910B01D5
:100AB000873709F0B3CF70E080EF92E0CF910C94CC
:100AC000360D81E0CF910C94940183E0FBCFCF9160
:100AD0000C948C0161E0E4CF80910A01CF910C94D9
:100AE000EE0281E080930A0199CF82E0FBCF83E0A0
:100AF000F9CF61E081E10E94CD1468EB7BE080E0FA
:100B000090E00E949F1360E081E1CBCF61E082E042
:100B10000E94CD1468EB7BE080E090E00E949F1380
:100B200060E082E0BECF60910C01C5CF8AE00E94F8
:100B3000EE02E8E9F3E0119283E0EC3FF807D9F721
:100B40006DCF62E370E080E090E00E949F134AE086
:100B500050E060910A0184E795E0CF910C947C17F6
:100B600060910A0180910901681731F04AE050E074
:100B700084E795E00E947C1780910A018093090127
:100B8000813020F0843058F1863090F18AE00E9464
:100B9000FB14892B79F484E00E94FB14019769F51A
:100BA00060E084E00E94CD1460ED77E080E090E0AA
:100BB0000E949F130E94F00442E069E08DE794E0F8
:100BC0000E9471098DE794E00E942A0880936204D4
:100BD00090910A01811116C0913089F508958BE832
:100BE00093E00E9471078BE893E00E942607CECF26
:100BF0008BE893E00E942B07C9CF80910A010E94E5
:100C0000EE02D8CF8130D9F4913019F482E080938C
:100C10000A0161E081E10E94CD1460E777E180E0A4
:100C200090E00E949F1360E081E10E94CD146CE28D
:100C300071E080E090E00E949F1310926204809126
:100C40000A0190916204923019F08230E1F4089523
:100C5000823019F483E080930A0161E082E00E940F
:100C6000CD1460E777E180E090E00E949F1360E0A0
:100C700082E00E94CD146CE271E080E090E00E947E
:100C80009F131092620480910A01833011F40E9434
:100C9000530480910A01843031F48BE893E00E9480
:100CA0002B070C94ED030895FC0185E991E09183F5
:100CB000808312821382148215828AE090E09783E7
:100CC000868310860895FC01778366830895CF9309
:100CD000DF93EC011886E881F9810190F081E02D25
:100CE0000995882319F08885836088870E946E1390
:100CF0006A837B838C839D83DF91CF910895CF920C
:100D0000DF92EF92FF920F931F93CF93DF93EC014B
:100D100088858B7F8887E881F9810190F081E02DBB
:100D2000CE010995182F8885869581701817B9F01E
:100D30000E946E136A837B838C839D83888592E0F7
:100D400089278887888582FB882780F9DF91CF9162
:100D50001F910F91FF90EF90DF90CF9008950E9428
:100D60006E13CA80DB80EC80FD80AB01BC014C19A6
:100D70005D096E097F098E819F81B0E0A0E0481770
:100D800059076A077B07F0F2888581701817D1F23E
:100D90000E946E136A837B838C839D83888591E098
:100DA0008927846088870E946E1309851A852B85A0
:100DB0003C85601B710B820B930B6D877E878F8741
:100DC000988B0E946E1369877A878B879C87BACF2E
:100DD000FC01808581700895CF93DF93EC010E9420
:100DE000540681EA92E099838883198ADF91CF9132
:100DF0000895FC01618B0C94670690E080E00895F3
:100E00000895FC011382128289EA92E09183808323
:100E1000648341872287138608950F931F93CF938E
:100E20008C01C62FFC0164818DE794E00E94F108DB
:100E3000F80163856C2B8DE794E00E9483088DE7B1
:100E400094E0CF911F910F910C947409FC011386CB
:100E500060E00C940D0728E0FC01238760E00C940F
:100E60000D070F931F93CF938C01C62F64600E94D0
:100E70000D0781E090E00E94D8136C2F6B7FC801B2
:100E80000E940D0782E390E0CF911F910F910C9487
:100E9000D8131F93CF93DF93EC01162F0E940D07F9
:100EA000612FCE01DF91CF911F910C9431070F93E9
:100EB0001F93CF93DF938C01D62FC42F607F642BB9
:100EC0000E94490780E1D89FB00111246C2BC80112
:100ED000DF91CF911F910F910C94490740E00C9442
:100EE000570761E00E946E0780ED97E00C94D813DD
:100EF00062E00E946E0780ED97E00C94D813CF93C8
:100F0000DF93CDB7DEB728970FB6F894DEBF0FBEDC
:100F1000CDBF28E0EEE2F1E0DE01119601900D92E6
:100F20002A95E1F7FC012085241710F44FEF420FBA
:100F300050E0440F551F21E030E02C0F3D1F420FC1
:100F4000531FFA012081620F606828960FB6F8944B
:100F5000DEBF0FBECDBFDF91CF910C946E07FC01B9
:100F60006681262F246026836C600C946E0741E016
:100F70000E94570781E090E00895CF93DF93EC0142
:100F8000423018F08D8188608D834887222329F0B4
:100F9000413019F48D8184608D8362E370E080E0DC
:100FA00090E00E949F136B85CE010E940D0768EEB2
:100FB00073E080E090E00E949F1360E3CE010E9406
:100FC000490784E991E10E94D81360E3CE010E94B1
:100FD000490784E991E10E94D81360E3CE010E94A1
:100FE000490786E990E00E94D81360E2CE010E9492
:100FF00049076D816062CE010E946E0784E08E8396
:10100000CE010E94AF07CE010E94710782E08F835C
:1010100066E0CE010E946E07CE01DF91CF910C9465
:101020007807CF93DF93EC018DE794E00E94DF080F
:101030001D8220E04A856985CE01DF91CF910C9415
:10104000BD070C9411088091B1049091B204891BE2
:10105000990B08959091B2048091B1042FEF3FEF66
:10106000981748F4E92FF0E0ED54FB4F208130E071
:101070009F5F9093B204C9010895E091B2048091FA
:10108000B104E81730F4F0E0ED54FB4F808190E0BC
:1010900008958FEF9FEF08950895CF93DF93EC01AC
:1010A000E0918904F0918A043097F1F09091B204B4
:1010B0008091B1049817C0F090E0292F30E02617F6
:1010C000370754F4DE01A20FB31F4C912D543B4F50
:1010D000D9014C939F5FF1CF1092B2046093B10499
:1010E000CB01DF91CF910994DF91CF910895E091E9
:1010F0008B04F0918C04309729F010928F04109299
:101100008E0409940895CF93DF931F92CDB7DEB775
:10111000698320918D042223F9F020918E042032DE
:1011200058F021E030E0FC013383228390E080E03E
:101130000F90DF91CF91089580918F04E82FF0E018
:10114000E057FB4F998190838F5F80938F0480934A
:101150008E0481E090E0ECCF61E0CE0101960E9428
:10116000450AF7CFCF92DF92EF92FF920F931F9332
:10117000CF93DF937C01CB018A0120918D04222340
:1011800089F0EB016B01C40ED51ECC15DD0569F0AD
:101190006991D701ED91FC910190F081E02DC7019B
:1011A0000995F3CF642F0E94450AC801DF91CF91C2
:1011B0001F910F91FF90EF90DF90CF9008951092C4
:1011C000B2041092B10410928F0410928E040E9407
:1011D000880987E798E00E94710A8DE498E00C94F2
:1011E0006C0A81E080938D046093B00410928F04A8
:1011F00010928E0408950F93062F21E040918E04E3
:1012000060E974E08091B0040E94EE0910928F04AE
:1012100010928E0410928D040F9108954F925F9258
:101220006F927F92AF92BF92CF92EF92FF920F9305
:101230001F93CF93DF935C01F62ED42F2801390141
:10124000EE2019F10E94F108CE2DC43008F0C3E061
:10125000C150B8F028E0C29FC0011124A30192013F
:1012600004C056954795379527958A95D2F7B901C9
:10127000D501ED91FC910190F081E02DC50109951A
:10128000E7CF60E0C5010E94FB084D2FD13208F086
:1012900040E22C2D63EB74E08F2D0E94A609109282
:1012A000B2048093B104DF91CF911F910F91FF9011
:1012B000EF90CF90BF90AF907F906F905F904F90E6
:1012C0000895CF92EF920F931F93C22EE12C00E06E
:1012D00010E098010E940E091F910F91EF90CF909E
:1012E000089521E00C94610961E00C94FB08EDE79E
:1012F000F4E01382128288EE93E0A0E0B0E08483F1
:101300009583A683B78385EB92E0918380830895CC
:101310001092400581E080933E0510923D0561E00A
:1013200082E10E94CD1461E083E10E94CD14E9EBDB
:10133000F0E080818E7F808380818D7F808380E25A
:101340008093B80085E48093BC000895413208F092
:1013500043C0909140059111FCCF91E090934005DE
:1013600020933E052FEF2093D30410921805240FED
:101370002093170590933F0590913F05880F892B87
:1013800080933F0580913D05813009F510923D0520
:1013900080913F058093BB008091BC0083FDF8CF16
:1013A00085EC8093BC00809140058130E1F3809111
:1013B0001805841710F440911805A9E1B5E0962F9F
:1013C000FB018E2F891B841720F0842F089585EE52
:1013D000E8CF8D918193F5CF40E0F7CF0F93413265
:1013E00008F04BC0909140059111FCCF92E0909392
:1013F000400500933E059FEF9093D304109218058B
:1014000040931705362FA9E1B5E0FB019E2F931BF2
:10141000941770F110923F0590913F05880F892B2A
:1014200080933F0580913D05813029F510923D055F
:1014300080913F058093BB008091BC0083FDF8CF75
:1014400085EC8093BC00222321F0809140058230FE
:10145000D1F38091D3048F3F91F08091D3048032F7
:1014600081F08091D304803371F084E00F9108956E
:1014700091919D93CBCF85EEE4CF81E0F7CF80E0D3
:10148000F5CF82E0F3CF83E0F1CF2091F504260F72
:101490003327331F21323105ECF420914005FC0144
:1014A00090E080E0243069F082E00895A091F50496
:1014B0002191AC0149505B4FA40FB52FB11D2C9366
:1014C0000196861798F38091F504680F6093F504F0
:1014D00080E0089581E0089590933A05809339055E
:1014E000089590933C0580933B05089585ED809386
:1014F000BC008091BC0084FDFCCF10924005089593
:1015000085EC8093BC001092400508951F920F92C5
:101510000FB60F9211242F933F934F935F936F93C6
:101520007F938F939F93AF93BF93EF93FF9380919C
:10153000B900887F803609F44CC008F03FC088327B
:1015400009F4A8C018F5803109F49CC0B8F48823C8
:1015500009F4F9C0883009F495C0FF91EF91BF916B
:10156000AF919F918F917F916F915F914F913F913B
:101570002F910F900FBE0F901F901895883109F48E
:1015800089C0803251F78093D30415C0803409F4A8
:101590009EC048F48033B9F38833F9F68093D304BE
:1015A0000E94800ADACF803509F485C0883509F4B5
:1015B00096C0883491F60E94760ACFCF883909F414
:1015C0008CC038F5883729F050F4883611F0803710
:1015D00021F683E0809340051092D40457C08838E8
:1015E00009F47BC0803919F0803809F0B6CF8091BA
:1015F000D404803208F071C0E091D40481E08E0FF1
:101600008093D4048091BB00F0E0EB52FB4F8083C9
:101610003DC0803B39F0E0F4803A09F479C0883A63
:1016200009F09BCF84E0809340051092F60410925D
:10163000F504E0913B05F0913C0509958091F50496
:1016400081110FC081E08093F5041092F70409C066
:10165000803C09F476C0883C09F473C0883B09F0EB
:101660007CCFE091F60481E08E0F8093F604F0E0E9
:10167000E950FB4F80818093BB009091F6048091EC
:10168000F50429C080913F058093BB0085EC8093D1
:10169000BC0063CF9091180580911705981758F5F5
:1016A000E091180581E08E0F80931805F0E0E75E69
:1016B000FA4F8081E9CFE091180581E08E0F809389
:1016C00018058091BB00F0E0E75EFA4F80839091AF
:1016D0001805809117059817C8F285E8D8CFE091D2
:1016E000180581E08E0F809318058091BB00F0E013
:1016F000E75EFA4F808380913E0581115CCF81E0E7
:1017000080933D0584EA8093BC001092400525CF6C
:101710000E94800A8091D404803230F4E091D40495
:10172000F0E0EB52FB4F10826091D40470E0E09146
:101730003905F0913A0585ED94E009951092D404AD
:101740000CCF85ECE0CF1092D30435CF1F920F92CF
:101750000FB60F9211242F933F934F935F936F9384
:101760007F938F939F93AF93BF93EF93FF9380915A
:10177000420587FF27C01092850010928400809157
:1017800042058F5F8093420580914205082E000C30
:10179000990B209141052817190629F024F0809112
:1017A00042058C30DCF18091840090918500049694
:1017B00080329E4408F47BC0809184009091850023
:1017C000049677C080914205082E000C990B209159
:1017D00041052817190699F294F2E09142058E2FDF
:1017E000EE0F990BFC01EE0FFF1FE80FF91FED5BE9
:1017F000FA4F808186FFC3CFE09142058E2FEE0F16
:10180000990BFC01EE0FFF1FE80FF91FED5BFA4F7C
:10181000808160E08F730E94CD14B1CF209184004D
:1018200030918500E09142058E2FEE0F990BFC015F
:10183000EE0FFF1FE80FF91FED5BFA4F81819281D8
:10184000820F931F9093890080938800E091420556
:101850008E2FEE0F990BFC01EE0FFF1FE80FF91F03
:10186000ED5BFA4F808186FF11C0E09142058E2F1B
:10187000EE0F990BFC01EE0FFF1FE80FF91FED5B58
:10188000FA4F808161E08F730E94CD14FF91EF9138
:10189000BF91AF919F918F917F916F915F914F9188
:1018A0003F912F910F900FBE0F901F90189580E2DF
:1018B0009EE490938900809388008FEF8093420587
:1018C000E5CFFC01909141059C3098F481E0890FAF
:1018D000809341059083892F90E0FC01EE0FFF1F5C
:1018E000E80FF91FED5BFA4F8CED95E09283818351
:1018F00008958FEF80830895DF92EF92FF920F9308
:101900001F93CF93DF93EC01D62E7A018901888152
:101910008C3008F067C061E08D2D0E9491148881A1
:10192000282F30E0F901EE0FFF1FE20FF31FED5BF0
:10193000FA4F9D2D9F736081607C692B608320E24C
:1019400032E02E193F0937FF02C02D5F3F4F35951A
:10195000279535952795298320E639E0201B310B03
:1019600037FF02C02D5F3F4F359527953595279559
:101970002A832CE0622F0E94E717829FB001112476
:1019800030E020E0AB01420F531FFA01EE0FFF1FC2
:10199000E40FF51FED5BFA4F908196FD16C02F5FA7
:1019A0003F4F2C30310571F781110FC0109280002C
:1019B00082E0809381001092850010928400B19A99
:1019C00080916F00826080936F00E8818E2F90E09D
:1019D000FC01EE0FFF1FE80FF91FED5BFA4F80814E
:1019E000806480838881DF91CF911F910F91FF9058
:1019F000EF90DF90089520E639E040E252E00C9449
:101A00007C0CDC01EC91EC3080F511968C911197F7
:101A100028E830E0281B310987FD3395220F331F5A
:101A2000220F331F6217730784F012968C9128E5FA
:101A300032E0281B310987FD3395220F331F220F17
:101A4000331F621773070CF49B014FB7F8948E2F66
:101A500090E022503109FC01EE0FFF1FE80FF91F43
:101A6000ED5BFA4F328321834FBF0895AF92BF924F
:101A7000CF92DF92EF92FF920F931F93CF93DF935A
:101A8000EC01603282E078070CF03EC0653B7105E6
:101A900014F064EB70E0898148E8A42EB12CA81AF8
:101AA000B10887FDB394AA0CBB1CAA0CBB1C0B2C61
:101AB000000CCC08DD0877FF02C070E060E0072E64
:101AC000000C880B990B2A8108E512E0021B110912
:101AD00027FD1395000F111F000F111F012E000C81
:101AE000220B330B3F932F931F930F9314EBE12E95
:101AF000F12C00E010E020E030E0A9010E94831703
:101B00000F900F900F900F90CE01DF91CF911F910A
:101B10000F91FF90EF90DF90CF90BF90AF900C941B
:101B2000010DCF93CFB7F89480916A05811127C03A
:101B3000E0EAF0E08491E9E8F0E09491E82FF0E049
:101B4000EE0FFF1FEF53FF4FA591B491EC91E923E6
:101B500021F461E08AE00E94CD1461E08AE00E94F5
:101B600091148CB580618CBD8CB580648CBD61E0B6
:101B70008DE00E94911461E08BE00E9491148091AD
:101B80006A058F5F80936A05CFBFCF910895BC012E
:101B90006E5F7F4FDC01ED91FC910190F081E02DB3
:101BA00040E0099591E0811190E0892F08952091FE
:101BB0006905222381F03FB7F8942091690521300F
:101BC00069F42DB3209367054DB3209168052095E6
:101BD00024232DBB3FBF8CBD9DBD08953093670569
:101BE000FACF8EBD00000DB407FEFDCF8EB508956F
:101BF00080916905882361F09FB7F8942091690569
:101C000080916705213019F48DBB9FBF08958FBF68
:101C10000895CF92DF92EF92FF920F931F93CF938D
:101C2000DF937C01C42EE901D62E6894D7F880E5B5
:101C300091E00E94D70D60E0F70186850E94CD14E7
:101C4000CA948D2D0E94F10D0023A1F08FEF90E03A
:101C50009C0102C0220F331F0A95E2F789018D2DE6
:101C60000E94F10D902F9095288192238023892B3B
:101C7000888301E0C00FD11D0C1530F48D2D0E941A
:101C8000F10D89930F5FF8CF80E00E94F10D8883FA
:101C900061E0F70186850E94CD14DF91CF911F91FD
:101CA0000F91FF90EF90DF90CF900C94F80DFC0116
:101CB00087EC92E0918380836687478708950F932E
:101CC0001F93CF93DF93EC01062F142F80E591E053
:101CD0000E94D70D60E08E850E94CD14802F0E9457
:101CE000F10D812F0E94F10D61E08E850E94CD14CF
:101CF000DF91CF911F910F910C94F80DDF92EF922D
:101D0000FF920F931F93CF93DF937C01C62F042F75
:101D1000D22E132F80E591E00E94D70D60E0F701ED
:101D200086850E94CD148C2F0E94F10DCD2DD12FD0
:101D30000C0F1D2F111DC017D10721F089910E9492
:101D4000F10DF9CF61E0F70186850E94CD14DF9196
:101D5000CF911F910F91FF90EF90DF900C94F80DB1
:101D60001F93CF93DF93EC01162F80E591E00E9443
:101D7000D70D60E08E850E94CD14812F80680E946F
:101D8000F10D80E00E94F10D182F61E08E850E9418
:101D9000CD140E94F80D812FDF91CF911F910895EE
:101DA0000F9341110E94090E0F9108950F931F93F5
:101DB000CF93DF938C01D62FC42F0E94B00E482FF3
:101DC0004C2B6D2FC801DF91CF911F910F910C9477
:101DD0005F0E0F931F93CF93DF938C01D62FC42FE9
:101DE0000E94B00EC0954C2F48236D2FC801DF9183
:101DF000CF911F910F910C945F0ECF92DF92EF92D3
:101E0000FF920F931F93CF93DF93EC016B01142F7D
:101E1000790140E062E00E945F0E44E06AE0CE019A
:101E20000E945F0E40E864E1CE010E945F0E9601C1
:101E3000412F62E1CE010E947E0E43E062E0CE01BE
:101E40000E945F0E08E813E16AE0CE010E94B00E26
:101E500082FF1BC040E062E0CE010E945F0E64E49E
:101E6000CE010E94B00EF701808362E4CE010E9491
:101E7000B00EF701818380E0DF91CF911F910F9128
:101E8000FF90EF90DF90CF90089501501109E1F697
:101E900083E0F2CF0F931F93CF938C014FE062E06A
:101EA0000E945F0EC3E062E370E080E090E00E9479
:101EB0009F1362E0C8010E94B00E84FF02C0C150AF
:101EC00091F7CF911F910F910895CF93DF93EC017C
:101ED00068E20E94B00E982F9370933041F0482F23
:101EE000436068E2CE01DF91CF910C945F0EDF91E9
:101EF000CF910895CF93DF93EC0161E08E850E942E
:101F0000911461E08E850E94CD148F858F3F09F476
:101F100051C060E00E9491148F850E94FB14892BB0
:101F200009F048C061E08F850E94911460E08F85C0
:101F30000E94CD1482E090E00E94D81361E08F856A
:101F40000E94CD1462E370E080E090E00E949F1355
:101F500040E064E2CE010E945F0E40E066E2CE0106
:101F60000E945F0E46E268E4CE010E945F0E40E8E8
:101F700064E5CE010E945F0E49EA66E5CE010E944B
:101F80005F0E43E068E5CE010E945F0E48EE6AE511
:101F9000CE010E945F0E40E46AE2CE010E945F0E15
:101FA0004DE362E2CE010E945F0ECE01DF91CF9140
:101FB0000C94650FCE010E944A0FCACF3F924F92F8
:101FC0005F926F927F928F929F92AF92BF92CF92C9
:101FD000DF92EF92FF920F931F93CF93DF9300D086
:101FE000CDB7DEB73C01162F942E290180E0A11455
:101FF000B10411F0F5018081382C329490EF392230
:10200000380E40E062E0C3010E945F0E4FE768E0D7
:10201000C3010E945F0E40E864E1C3010E945F0EAD
:102020009201402F62E1C3010E947E0E432D6AE1BE
:10203000C3010E945F0E412F62E0C3010E945F0E48
:102040001C3029F440E86AE1C3010E94D60E00ED7D
:1020500017E068E0C3010E94B00E982F992109F0A3
:102060007BC080FD03C00150110999F783E038C09F
:10207000E114F10409F448C0C114D10409F444C0C6
:1020800064E1C3010E94B00EF6019081981708F434
:102090005FC08083082D9701482F62E1C3010E9431
:1020A000D00E68E1C3010E94B00E8770A114B10484
:1020B00011F0F501808313FD4DC0E114F10409F422
:1020C00045C0C114D10409F441C09E899923F1F19E
:1020D000F60140814130D1F4843009F047C08FEFE0
:1020E0000F900F90DF91CF911F910F91FF90EF9084
:1020F000DF90CF90BF90AF909F908F907F906F9028
:102100005F904F903F90089580E0D5CF423070F1BE
:1021100081112CC042509E012F5F3F4FB701C30178
:102120000E94FD0E8111DCCFF6018081E80EF11CCA
:10213000F701329790818981981318C0F1E0EF1A66
:10214000F108F70190818A81981310C080E0C8CF10
:1021500084E0C6CF82E0C4CF6CE0C3010E94B00E21
:10216000182F837109F484CF81E0BACF87E0B8CF0C
:102170008F92AF92BF92CF92DF92EF92FF920F9326
:102180001F93AF928C2C570168017901042F9B019A
:1021900040E36CE00E94DE0F0F901F910F91FF90C3
:1021A000EF90DF90CF90BF90AF908F9008952F92D7
:1021B0003F924F925F926F927F928F929F92AF92D7
:1021C000BF92CF92DF92EF92FF920F931F93CF9324
:1021D000DF93CDB7DEB72D970FB6F894DEBF0FBEF5
:1021E000CDBF16E0413508F045C1342E4B013C010E
:1021F00040E86CE10E94E90E83E98983332029F0ED
:1022000081E0F4019081953008F480E02224239449
:10221000B12C9B2D990F990F990FD32CD91AD7FC5C
:10222000D12C32E0882319F098E89B8333E021E039
:102230009D2D977009F420E09D2D95959595959588
:10224000290FC9F094E0811193E0291708F4922F27
:10225000EB2DF0E03196E80DF91D232F4191A1E01F
:10226000B0E0AC0FBD1FA20FB11D4C932F5F422FEA
:10227000431B491798F3882311F0F8E0DF0E8FE134
:102280008D150CF082C090E79A838B819C81892701
:102290009D8189279E8189278F839E01285F3F4FDB
:1022A00047E0BE016F5F7F4FC3010E94FD0E182FF4
:1022B0008111E0C01B86E3E0EA87DC86CE01079649
:1022C0002C0199E09D87CB844C2D4295407F4C0D8D
:1022D0006AE1C3010E945F0EA12CCE010B967C0126
:1022E0008E01065F1F4F92014D85BE016F5F7F4FCC
:1022F000C3010E94B810182F823009F065C06CE14C
:10230000C3010E94B00E85FDB5C08F7109F480E253
:10231000282F30E04D2DDD0C550B421753070CF0E4
:102320009DC0D82EE82FE595E595E595EF5F982FB0
:10233000977081E009F480E0E80F81E090E08C0F75
:102340009D1F8E0F911DFC012150310927703327ED
:1023500081E090E002C0880F991F2A95E2F79C0166
:102360008081822B80838BCF85E98983332031F074
:1023700081E0F4019081983008F04BCF80E049CFA4
:1023800087E9898326E0B22EF9CF9D2D97709B8730
:102390008D2D8595859585958E5F282F2295207F9B
:1023A000290F2A8321E0911101C020E0280F2D87F9
:1023B00044244394512C4C0E5D1E480E511CE9E000
:1023C000E81BEA87DC867FCF811154C080E2D82EDB
:1023D0009C8590320CF457CF8B81883809F040C02F
:1023E00083E093E0EB2DF0E03196E80DF91D980FB6
:1023F000A1E0B0E0AC0FBD1FA80FB11D2C9121933F
:102400008F5F8913F5CFBA84E3E0BE124DC08B8590
:1024100081114AC09E012D5F3F4F41E0B201C301CF
:102420000E94FD0E182F811125C09B81F201818130
:1024300098133CC09C818281981338C0808182FFB0
:1024400012C02394F2E02F1609F48ECF83E02816F1
:1024500009F496CF91E0291609F4CECE15E00AC012
:1024600082E094E0BFCFF4018387822D880F820D34
:102470008F5F8083812F2D960FB6F894DEBF0FBE3D
:10248000CDBFDF91CF911F910F91FF90EF90DF9023
:10249000CF90BF90AF909F908F907F906F905F9004
:1024A0004F903F902F90089511E0E4CF17E0E2CFD6
:1024B0004F925F926F927F928F929F92AF92CF9244
:1024C000EF92FF920F931F93CF93DF9300D0CDB77E
:1024D000DEB76A8341155105B9F1F90160816230B7
:1024E00098F149012A013C0140E86CE10E94E90EA3
:1024F00087E08983A12CC12CCE0101967C01840147
:10250000920141E0BE016E5F7F4FC3010E94B8108F
:10251000811109C0F40180818230C1F481E0998188
:10252000911101C080E00F900F90DF91CF911F912A
:102530000F91FF90EF90CF90AF909F908F907F90F2
:102540006F905F904F90089584E0EDCF81E0EBCFE6
:102550009A01AB0166E20C9458120F931F93CF932C
:10256000DF9300D01F92CDB7DEB78C0182E08B8362
:1025700040E064E2C8010E945F0E40E066E2C801EC
:102580000E945F0E46E268E4C8010E945F0EAE0141
:102590004D5F5F4FBE016F5F7F4FC8010E94A81261
:1025A000982F9D7F81E009F080E00F900F900F90B1
:1025B000DF91CF911F910F9108958F929F92AF92CB
:1025C000CF92EF92FF920F931F93CF93DF9300D0A0
:1025D00000D0CDB7DEB74C0180E589831A829E0119
:1025E0002D5F3F4F42E0BE016F5F7F4FC4010E94ED
:1025F000FD0E811116C0A12CC12CF12CE12C10E094
:1026000000E030E020E044E0BE016F5F7F4FC40196
:102610000E94B810833021F0811103C081E001C015
:1026200080E00F900F900F900F90DF91CF911F914E
:102630000F91FF90EF90CF90AF909F908F90089563
:1026400048E060E10C94E90E1F920F920FB60F92D2
:1026500011242F933F938F939F93AF93BF938091B8
:10266000700590917105A0917205B091730530913C
:102670006F0526E0230F2D3768F129E8230F039615
:10268000A11DB11D20936F05809370059093710576
:10269000A0937205B093730580916B0590916C05C2
:1026A000A0916D05B0916E050196A11DB11D80939D
:1026B0006B0590936C05A0936D05B0936E05BF916B
:1026C000AF919F918F913F912F910F900FBE0F90DF
:1026D0001F9018950296A11DB11DD4CF2FB7F89465
:1026E00060917005709171058091720590917305EC
:1026F0002FBF08953FB7F89480916B0590916C05BA
:10270000A0916D05B0916E0526B5A89B05C02F3F21
:1027100019F00196A11DB11D3FBFBA2FA92F982F07
:102720008827BC01CD01620F711D811D911D43E001
:10273000660F771F881F991F4A95D1F708958F92CA
:102740009F92AF92BF92CF92DF92EF92FF926B0176
:102750007C010E947A134B015C01C114D104E10495
:10276000F104E9F00E94D6170E947A1368197909DA
:102770008A099B09683E73408105910570F321E049
:10278000C21AD108E108F10888EE880E83E0981E8D
:10279000A11CB11CC114D104E104F10429F7FF907C
:1027A000EF90DF90CF90BF90AF909F908F90089563
:1027B000000000008330910528F0880F991F0597CD
:1027C0000197F1F70895789484B5836084BD85B549
:1027D000836085BDEEE6F0E0808181608083E1E882
:1027E000F0E082E08083808181608083E0E8F0E037
:1027F000808181608083E1EBF0E080818460808370
:10280000E0EBF0E080818160808386E880937A004D
:102810001092C10008951F93CF93DF93182FEB01FF
:1028200061E00E949114209739F460E0812FDF91DC
:10283000CF911F910C94CD14CF3FD10511F461E0DD
:10284000F5CFE12FF0E0E859FF4FE491E43031F1AA
:1028500040F4E230B1F0E330E1F0C038D1057CF76C
:10286000E4CFE83029F1E93059F1E530B1F7809152
:102870008000806280938000D0938B00C0938A0098
:1028800004C084B5806884BDC7BDDF91CF911F911E
:10289000089584B5806284BDC8BDF7CF8091800063
:1028A000806880938000D0938900C0938800EDCF2A
:1028B0008091B00080688093B000C093B300E5CFF2
:1028C0008091B00080628093B000C093B400DDCFEF
:1028D000843081F028F48230E9F08330F9F00895F3
:1028E000883071F0893091F08530B9F480918000A2
:1028F0008F7D03C0809180008F7780938000089542
:102900008091B0008F778093B00008958091B000DF
:102910008F7DF9CF84B58F7784BD089584B58F7D81
:10292000FBCFCF93DF9390E0FC01E158FF4F249160
:102930008A569F4FFC0184918823C9F090E0880F4C
:10294000991FFC01EF53FF4FA591B491FC01E9548D
:10295000FF4FC591D49161110DC09FB7F8948C9130
:10296000209582238C938881282328839FBFDF9121
:10297000CF910895623051F49FB7F8943C91822F23
:10298000809583238C93E8812E2BEFCF8FB7F8941B
:10299000EC912E2B2C938FBFEACF1F93CF93DF9315
:1029A000282F30E0F901E859FF4F8491F901E158EF
:1029B000FF4FD491F901EA56FF4FC491CC23A9F0FF
:1029C000162F81110E946814EC2FF0E0EE0FFF1F0C
:1029D000E954FF4FA591B4918FB7F894EC91111180
:1029E00008C0D095DE23DC938FBFDF91CF911F917C
:1029F0000895DE2BF8CFCF93DF93282F30E0F90135
:102A0000E859FF4F8491F901E158FF4FD491F90142
:102A1000EA56FF4FC491CC23A1F081110E946814A3
:102A2000EC2FF0E0EE0FFF1FE355FF4FA591B4919F
:102A3000EC91ED2381E090E009F480E0DF91CF910B
:102A4000089580E090E0FACFFC01918D228D892FCE
:102A500090E0805C9F4F821B91098F7399270895A6
:102A6000FC01918D828D981731F0828DE80FF11D58
:102A7000858D90E008958FEF9FEF0895FC01918D73
:102A8000828D981761F0A28DAE0FBF2FB11D5D969C
:102A90008C91928D9F5F9F73928F90E008958FEF3E
:102AA0009FEF0895FC01538D448D252F30E0842F36
:102AB00090E0821B930B541710F0CF960895019766
:102AC000089581EA96E1892B49F080E090E0892B16
:102AD00029F00E94A11681110C9400000895FC01B8
:102AE000A48DA80FB92FB11DA35ABF4F2C91848D6F
:102AF00090E001968F739927848FA689B7892C93CC
:102B0000A089B1898C9180648C93938D848D981366
:102B100006C00288F389E02D80818F7D808308952F
:102B2000CF93DF93EC01888D8823B9F0AA89BB8904
:102B3000E889F9898C9185FD03C0808186FD0DC0EF
:102B40000FB607FCF7CF8C9185FFF2CF808185FF10
:102B5000EDCFCE010E946F15E9CFDF91CF9108959F
:102B6000EF92FF920F931F93CF93DF93EC0181E0DD
:102B7000888F9B8D8C8D981316C0E889F989808188
:102B800085FF11C0EE89FF896083E889F98980811A
:102B90008064808381E090E0DF91CF911F910F915D
:102BA000FF90EF900895F62E0B8D10E00F5F1F4FF2
:102BB0000F731127E02E8C8D8E110CC00FB607FC01
:102BC000FACFE889F989808185FFF5CFCE010E948F
:102BD0006F15F1CFEB8DEC0FFD2FF11DE35AFF4F79
:102BE000F0820B8FEA89FB8980818062D2CFCF92FD
:102BF000DF92EF92FF921F93CF93DF93EC016A0174
:102C00007B01122F60E874E88EE190E0A701960145
:102C10000E94F317215031094109510956954795F2
:102C200037952795E889F98982E08083211580E12D
:102C3000380798F0E889F989108260E472E48FE03F
:102C400090E0A70196010E94F31721503109410934
:102C500051095695479537952795EC85FD85308325
:102C6000EE85FF852083188EEC89FD891083EA8923
:102C7000FB89808188698083EA89FB8980818F7DD7
:102C80008083DF91CF911F91FF90EF90DF90CF90E5
:102C900008951F920F920FB60F9211242F938F93C6
:102CA0009F93EF93FF93E0918405F09185058081D8
:102CB000E0918A05F0918B0582FD1BC09081809187
:102CC0008D058F5F8F7320918E05821741F0E09103
:102CD0008D05F0E0EC58FA4F958F80938D05FF91AC
:102CE000EF919F918F912F910F900FBE0F901F909A
:102CF00018958081F4CF1F920F920FB60F92112476
:102D00002F933F934F935F936F937F938F939F93F3
:102D1000AF93BF93EF93FF9384E795E00E946F1505
:102D2000FF91EF91BF91AF919F918F917F916F91A3
:102D30005F914F913F912F910F900FBE0F901F9079
:102D4000189584E795E00E94241521E0892B09F469
:102D500020E0822F0895E4E7F5E01382128288EEE6
:102D600093E0A0E0B0E084839583A683B78381EDF0
:102D700092E09183808385EC90E09587848784EC52
:102D800090E09787868780EC90E0918B808B81EC38
:102D900090E0938B828B82EC90E0958B848B86EC19
:102DA00090E0978B868B118E128E138E148E089561
:102DB000AF92BF92CF92DF92EF92FF920F931F9349
:102DC000CF93DF936C017B018B01040F151FEB0187
:102DD0005E01AE18BF08C017D10759F06991D6013E
:102DE000ED91FC910190F081E02DC6010995892BB0
:102DF00079F7C501DF91CF911F910F91FF90EF906F
:102E0000DF90CF90BF90AF900895FB01019000201C
:102E1000E9F73197AF01461B570BDC01ED91FC91AF
:102E20000280F381E02D09946115710511F00C9475
:102E3000051790E080E00895DC01ED91FC91019090
:102E4000F081E02D09948F929F92AF92BF92EF9202
:102E5000FF920F931F93CF93DF93CDB7DEB7A19768
:102E60000FB6F894DEBF0FBECDBF7C01FA01CB01D7
:102E700019A2223008F42AE08E010F5D1F4F822E26
:102E8000912CB12CA12CBF01A50194010E94F31734
:102E9000F901CA016A300CF5605DD8016E938D01AD
:102EA000232B242B252B79F790E080E0109721F03D
:102EB000BD01C7010E940517A1960FB6F894DEBFA9
:102EC0000FBECDBFDF91CF911F910F91FF90EF907B
:102ED000BF90AF909F908F900895695CDECF2115D1
:102EE000310541F4DC01ED91FC910190F081E02D80
:102EF000642F09940C9423179A01462F50E070E038
:102F000060E00C946F174F925F926F927F92AF9236
:102F1000BF92CF92DF92EF92FF920F931F93CF93C6
:102F2000DF93CDB7DEB729013A019B01AC0124192B
:102F300035094609570989899A89AB89BC89BC0139
:102F4000CD016A197B098C099D090E94D717A80138
:102F5000970124193509460957090E941518CA0115
:102F6000B9016A0D7B1D8C1D9D1DDF91CF911F91B5
:102F70000F91FF90EF90DF90CF90BF90AF907F9038
:102F80006F905F904F9008950E94541808950E948A
:102F9000E3130E94C6170E94DB00C1E6D5E10E9440
:102FA000B0052097E1F30E946115F9CF0895DB0188
:102FB0008F939F930E943A18BF91AF91A29F800D6B
:102FC000911DA39F900DB29F900D11240895991B00
:102FD00079E004C0991F961708F0961B881F7A9510
:102FE000C9F780950895A1E21A2EAA1BBB1BFD010B
:102FF0000DC0AA1FBB1FEE1FFF1FA217B307E407D8
:10300000F50720F0A21BB30BE40BF50B661F771F2F
:10301000881F991F1A9469F760957095809590950F
:103020009B01AC01BD01CF010895052E97FB1EF455
:1030300000940E942C1857FD07D00E94F31707FC3C
:1030400003D04EF40C942C18509540953095219552
:103050003F4F4F4F5F4F08959095809570956195C4
:103060007F4F8F4F9F4F0895EE0FFF1F0590F491F4
:10307000E02D09940E944518A59F900DB49F900DD6
:10308000A49F800D911D11240895A29FB001B39FAC
:10309000C001A39F700D811D1124911DB29F700D61
:1030A000811D1124911D089581E090E0F8940C9405
:1030B0006918FB01DC018D91019080190110D9F391
:1030C000990B0895FB01DC0101900D920020E1F7BE
:0630D0000895F894FFCF03
:1030D6009F01F301260258020501013C8C2741633A
:1030E6006365737320436F64653F00000000008AC8
:1030F60037F280415447434741415441470000005D
:103106004000140054004163636573730041757495
:10311600686F72697A65642100436F6E67726174C5
:10312600756C6174696F6E73210044656E696564C0
:1031360021002020202020202020202020202020A8
:1031460020200048656C70202D2050757A7A6C65B9
:103156002000437573746F6D204D657373616765E9
:103166000000000000C4170000000097009300490B
:1031760064656E746966792074686520636F6D6D29
:103186006F6E20444E412073657175656E636520D0
:103196006265747765656E20746865203220766195
:1031A6007269616E747320796F7520686176652027
:1031B600646973636F766572656420736F206661F8
:1031C600722E00416E616C797A696E67207468654B
:1031D60020636F6D706F736974696F6E206F662000
:1031E60074686520766972757320697320746865E2
:1031F600206B65792E005265636F6E737469747502
:10320600746520436F7669642D3139207370726559
:103216006164696E672061726F756E64207468659B
:1032260020776F726C642E0052656D656D626572F3
:103236002074686520436F7669642D31392070618A
:103246006E64656D69632070686173657320776568
:103256002068617665206265656E207468726F7598
:1032660067682E00414354475F14071508000000A5
:10327600009700930000000000B707D816FD06006F
:1032860007000000008308B208FD064C0823082A40
:10329600083D0800000000D710AD12C70D00000061
:1032A60000B015D8165215901524153E1530150088
:00000001FF
